:100000006429B200F839A400A40CA40C240C8407C1
:100010007320B20000055F293208031C03010006AB
:10002000320580065F29A01123080319A0150530A9
:10003000A2002730A900103029200330A900E830A1
:100040002920A90164302920A9010A3029202C087F
:100050003028A8002D08A5002C08A400FA202408A8
:10006000A400A2030319A011230803193A282202AD
:10007000031841282408031DA011A0194128303E6F
:10008000472808000C1E4228990003145F292119F3
:100090004228080083169B0083161C141A089B0A2A
:1000A0005F29A901A800FF30A807031CA907031CAA
:1000B0005F290330A500E5305F205328A501F63EF7
:1000C000A400A509031C6A28FE300000A407031839
:1000D0006528A4070000A50F6428000024187028D4
:1000E00024187228080000308A0032080739820775
:1000F0000134023404340834103420344034803461
:1001000027082F068039B100A71F9128A409A50947
:10011000A609A709A40A0319A50A0319A60A03191F
:10012000A70AAF1F9E28AC09AD09AE09AF09AC0AFA
:100130000319AD0A0319AE0A0319AF0AA801A901F0
:10014000AA01AB01B601B701B801B9012F082E040D
:100150002D042C040319DC282030B0000310A40D5A
:10016000A50DA60DA70DB60DB70DB80DB90D2F082D
:100170003902031DC5282E083802031DC5282D0885
:100180003702031DC5282C083602031CD6282C086C
:10019000B6022D08031C2D0FB7022E08031C2E0FCC
:1001A000B8022F08031C2F0FB9020314A80DA90DC4
:1001B000AA0DAB0DB00BAE28B11FE928A809A909FB
:1001C000AA09AB09A80A0319A90A0319AA0A03195B
:1001D000AB0A3608AC003708AD003808AE00390865
:1001E000AF002808A4002908A5002A08A6002B08AB
:1001F000A7005F29AD01AC011030B000250DAC0D9A
:10020000AD0D2808AC022908031C290FAD02031804
:1002100010292808AC0729080318290FAD07031077
:10022000A40DA50DB00BFE2824085F292030B000D6
:10023000B601B701B801B9010310241C2D292C08FF
:10024000B6072D0803182D0FB7072E0803182E0F19
:10025000B8072F0803182F0FB907B90CB80CB70C43
:10026000B60CA70CA60CA50CA40CB00B1C290800FE
:100270001030B300A501A401B10CB00C031C462939
:100280002808A40729080318290FA507A50CA40C02
:10029000AD0CAC0CB30B3C292C085F29A400A71BA8
:1002A000532124085F29A409A509A609A709A40ABE
:1002B0000319A50A0319A60A0319A70A080083133C
:1002C000831203130000080083160F3099002030BA
:1002D0009800831280309800A00142308316860077
:1002E000FD308500073083129F00982A64305E201D
:1002F000861564305E20061464305E2086116430FA
:100300005E20061064305E2008007621851464307B
:100310005E20D221E421061BC1298519AF294D3069
:10032000422041304220473042204E30422045306A
:100330004220543042203D304220203042200430C0
:10034000A100A3013B08AD003A08AC001320203007
:1003500042204220422042200D304220C0294D3010
:100360003A07C2003B080318013EC3004D3042204B
:100370003A0842203B0842204208422043084220DB
:100380008B29051DC929061086150A3051208611B2
:100390000800852985100A305E20080085140A307F
:1003A0005E2008000B30C100CA21CE213A30840003
:1003B0004108003E01200310051803140C200130F1
:1003C000C1020318D4290800CA21CE2183100518C0
:1003D000831483184014831C4010CA21CE2183103B
:1003E000051883148318C014831CC010CA21CE21A1
:1003F00083100518831483184015831C4011CA21EB
:10040000CE218310051883148318C015831CC011D6
:10041000CA21CE2183100518831483184016831C2B
:100420004012CA21CE218310051883148318C016E8
:10043000831CC012861514305E200800560855042F
:10044000031D232A0800A701A6013B08A5003A08BE
:10045000A400AF01AE011030AD00AC011621270899
:10046000DA002608D9002508D8002408D7005A0841
:10047000A7005908A6005808A5005708A400AF0116
:10048000AE015608AD005508AC0080202708DA0000
:100490002608D9002508D8002408D7005808BB0032
:1004A0005708BA0010303B02031C5A2A0F30BB0019
:1004B000FF30BA0008003B08B1003A08B000A901BB
:1004C0002D30A8003821C7002D08C8004808C500F5
:1004D000C6010310C50C4708C90001304805CA0011
:1004E0004A08B1004908B000A9010A30A800382123
:1004F000C9002D08CA004A08CB00CC010310CB0C60
:100500004908C70001304A05C80001304802031CF1
:10051000972A4B08093A4C04031D942AC50A03196B
:10052000C60ACC01CB01972ACB0A0319CC0A0800D2
:1005300006100330A900E8305220CF01CE01CD01D2
:10054000861300304A20C40001304A20D5004C20D8
:10055000D60003304A20DB004C20DC0086158514D1
:10056000BB01BA0114305E200519B72A8521861116
:1005700014305E20D2211E228618E32A3B08AD00EB
:100580003A08AC00AE01AF01013EBC00F030BD0046
:100590002D0803182D0FBD07FF30BE002E080318CD
:1005A0002E0FBE07FF30BF002F0803182F0FBF0705
:1005B0003F08A7003E08A6003D08A5003C084E21C4
:1005C000BA002508BB0002304F02031CF32A4E0874
:1005D000A5004D08A400A9014F08A800FA20D100E9
:1005E0002508D200F72A4E08D2004D08D1003B085A
:1005F0005202031C0A2B031D012B3A085102031C53
:100600000A2B3A085102D3003B08031C013E520258
:10061000D400122B51083A02D3005208031C013EA9
:100620003B02D400D408031D192B0A305302031CCB
:10063000202B3B08CE003A08CD000130CF002B2BF9
:100640000F304F0203182B2B3A08CD073B08031835
:10065000013ECE07CF0AE42101305120C01D322BCC
:100660000612342B06160616401E382B86123A2B1D
:1006700086168616061BD62B8519982B5B22C40876
:10068000031D6B2B413042205A304220493042201A
:100690004D304220553042205430422048304220D4
:1006A000203042203D304220203042200430A10042
:1006B000A3014608AD004508AC0013202E304220AF
:1006C000A3014C08AD004B08AC00132020304220A1
:1006D0000D304220972B453042204C30422045308F
:1006E000422056304220413042205430422049308E
:1006F00042204F3042204E304220203042203D30B8
:100700004220203042200430A100A3014608AD0061
:100710004508AC0013202E304220A3014C08AD0048
:100720004B08AC001320203042200D304220D32B48
:10073000C408031DB62B41304D07B4004E08031802
:10074000013EB5004F083407C20035080318013ECA
:10075000C300413042204D0842204E0842204F083D
:1007600042204208422043084220D02B45304D070A
:10077000B4004E080318013EB5004F083407C2000C
:1007800035080318013EC300453042204D08422081
:100790004E0842204F08422042084220430842208F
:1007A000CF01CE01CD01061BD62BD32BAE2A630081
:0207B000D72B45
:02400E00223F4F
:0A42000000004A000B00000010004F
:00000001FF
